:020000040000FA
:020000000528D1
:08000800112A07309F00831646
:100010009F018501860107308100831285018601D9
:100020003D3081001430A3008B178B16A601A70169
:10003000A801A901AA01AB01A201FC2126083420D4
:1000400022082E20860000220422042204220422F8
:10005000A20A2208053C031D20281C2882075B28D1
:100060005D285F28612863288207652870287B281F
:10007000862891289C28A728B228BD28C828D328DC
:10008000DE28E928F428FF280A29152920292B2908
:10009000362941294C29572962296D297829832934
:1000A0008E299929A429AF29BA29C529D029DB2964
:1000B000E629F12916282708080028080800290839
:1000C00008002A0808002B0808007C30A7008230AE
:1000D000A8008230A9008230AA007C30AB00080062
:1000E0000030A7008430A800FE30A9008030AA00AC
:1000F0000030AB0008008430A700C230A800A23056
:10010000A9009230AA008C30AB0008004430A70050
:100110008230A8009230A9009230AA006C30AB0067
:1001200008001030A7001830A8001430A900FE30D5
:10013000AA001030AB0008005E30A7009230A80083
:100140009230A9009230AA006230AB0008007C30E7
:10015000A7009230A8009230A9009230AA00643023
:10016000AB0008008230A7004230A8002230A9006E
:100170001230AA000E30AB0008006C30A70092309D
:10018000A8009230A9009230AA006C30AB000800A1
:100190004C30A7009230A8009230A9009230AA00FB
:1001A0007C30AB000800FC30A7001230A8001230F1
:1001B000A9001230AA00FC30AB000800FE30A700F6
:1001C0009230A8009230A9009230AA006C30AB00A7
:1001D00008007C30A7008230A8008230A90082305D
:1001E000AA004430AB000800FE30A7008230A8000F
:1001F0008230A9008230AA007C30AB000800FE30BB
:10020000A7009230A8009230A9009230AA00823054
:10021000AB000800FE30A7001230A8001230A90081
:100220001230AA000230AB0008007C30A7009230E8
:10023000A8009230A9009230AA007430AB000800E8
:10024000FE30A7001030A8001030A9001030AA001E
:10025000FE30AB0008000030A7008230A800FE305E
:10026000A9008230AA000030AB0008007030A7005F
:100270008030A8008030A9008030AA007E30AB001A
:100280000800FE30A7001030A8002830A900443034
:10029000AA008230AB000800FE30A7008030A80022
:1002A0008030A9008030AA008030AB000800FE300A
:1002B000A7000430A8001830A9000430AA00FE30BE
:1002C000AB000800FE30A7000830A8001030A900DD
:1002D0002030AA00FE30AB000800FA30A700123030
:1002E000A8002230A9004230AA00FA30AB00080072
:1002F0007C30A7008230A8008230A9008230AA009A
:100300007C30AB000800FE30A7001230A80012308D
:10031000A9001230AA000C30AB0008007C30A70006
:100320008230A800A230A9004230AA00BC30AB0045
:100330000800FE30A7001230A8003230A900523069
:10034000AA008C30AB0008004C30A7009230A80007
:100350009230A9009230AA006430AB00080002304D
:10036000A7000230A800FE30A9000230AA00023027
:10037000AB0008007E30A7008030A8008030A900C4
:100380008030AA007E30AB0008003E30A70040302D
:10039000A8008030A9004030AA003F30AB00080020
:1003A000FE30A7004030A8003030A9004030AA003D
:1003B000FE30AB000800C630A7002830A80010307F
:1003C000A9002830AA00C630AB0008000630A700FC
:1003D0000830A800F030A9000830AA000630AB00B1
:1003E0000800C230A700A230A8009230A9008A30CD
:1003F000AA008630AB00080085140C228510080086
:1004000005150C22051108000F30A000A100A10B5A
:10041000072AA00B062A0800FA30A100A10B0E2A19
:100420000800A400030EA5003D308100A30B1B2A89
:10043000A60A1430A300250E8300A40E240E0B116F
:020440000900B1
:02400E00293F48
:00000001FF
